:100000000C94CE030C9406040C9406040C94060481
:100010000C9406040C9406040C9406040C94060438
:100020000C9406040C9406040C9406040C94642DA1
:100030000C94132E0C9425280C9406040C9406049E
:100040000C9406040C9406040C9406040C94AE283C
:100050000C9406040C9406040C9406040C940604F8
:100060000C9406040C9406040C9406040C940604E8
:100070000C940604AF06AF06DB06DB063C0733082C
:10008000330833085A07C207D307D307CC13CF135B
:10009000D413D913DE13E313E813ED13F213F8139B
:1000A000FD139E211022A62170217421AA217721FF
:1000B000AD21B821822106228621BC218A21C021BE
:1000C000EA218E21C421F4219421CA21D4217B214B
:1000D000B1217E21B4219921CF21E02100220222E9
:1000E0006C21A2211922CB23D123BF23C523D723DF
:1000F000DD23E3236D257025A725BA25C225CD254F
:10010000D025D025D02518261826D525D825DD259B
:10011000EA25F725FA25FE250B267B2EA22E9A2FFF
:10012000A22E9A2FEE2E112F9A2F682F772F2900AB
:100130001E001F00200021002200230024002500B3
:10014000260027002D002E0031002B0014001A007D
:100150000800150017001C0018000C001200130006
:100160002F0030003100390004001600070009009C
:100170000A000B000D000E000F0033003400640075
:100180002800E10032001D001B00060019000500D8
:10019000110010003600370038000000E500E000D4
:1001A000E3000000E2002C002C002C00E600E70039
:1001B00000006500215200002A00007C3A003B004C
:1001C0003C003D003E003F00400041004200430033
:1001D000440045000100010001005200010001003F
:1001E0000100010001000100010001000100010007
:1001F00001000100500051004F000100010001000A
:1002000001000100010001000100010001000100E6
:1002100001000100010001000100010001000100D6
:1002200001000100010001000100010001000100C6
:1002300001000100010001000100010001000100B6
:10024000010001004C00010001000100010001005B
:100250000100010001000100010001000100010096
:100260000100010001000100010001000100010086
:100270000100010001000100010001000100010076
:100280000100010001000100010001000100010066
:100290000100010001000100010001000100010056
:1002A0000100010001000100010001000100010046
:1002B0000100010001000100010001000100010036
:1002C0000100010001000100010001000100010026
:1002D0000100010001000100010001000100010016
:1002E0000100010001000100010001000100010006
:1002F00001000100010001000100010001000100F6
:1003000001000100010001000100010001000100E5
:1003100001000100010001000100010001000100D5
:1003200001000100010001000100010001000100C5
:1003300001000100010001000100010001000100B5
:1003400001000100010001000100010001000100A5
:1003500001000100010001000100010001001E0F69
:100360000500047F3F1F643214643214783C1E1E63
:10037000140A052223252628292A2C2D2F30323332
:100380003536383A3B3D3E4042434547494A4C4E5C
:100390005051535557595A5C5E6062646668696B88
:1003A0006D6F71737577797B7D7F81838587898A8E
:1003B0008C8E90929496989A9C9E9FA1A3A5A7A894
:1003C000AAACAEAFB1B3B4B6B8B9BBBCBEBFC1C2C4
:1003D000C3C5C6C7C9CACBCCCDCED0D1D2D2D3D457
:1003E000D5D6D7D7D8D9D9DADADBDBDBDCDCDCDC75
:1003F000DCDDDDDDDDDCDCDCDCDCDBDBDBDADAD943
:10040000D9D8D7D7D6D5D4D3D2D2D1D0CECDCCCBC4
:10041000CAC9C7C6C5C3C2C1BFBEBCBBB9B8B6B4E2
:10042000B3B1AFAEACAAA8A7A5A3A19F9E9C9A9872
:10043000969492908E8C8A89878583817F7D7B7943
:10044000777573716F6D6B6968666462605E5C5A24
:100450005957555351504E4C4A4947454342403EE7
:100460003D3B3A3836353332302F2D2C2A29282679
:10047000252322FFAA7F554000010101010101014E
:100480000101020202020202020202030303030349
:100490000303030404040404040405050505050618
:1004A00006060606070707070708080808090909D6
:1004B000090A0A0A0B0B0B0C0C0C0D0D0D0E0E0E7F
:1004C0000F0F0F1010111111121213131414151510
:1004D00016161717181819191A1A1B1B1C1D1D1E82
:1004E0001E1F2020212222232424252626272829D6
:1004F000292A2B2C2D2D2E2F303132323334353604
:100500003738393A3B3C3D3E3F4041424344454603
:100510004748494A4C4D4E4F5051535455565859DF
:100520005A5B5D5E5F616264656668696B6C6D6F86
:100530007072737577787A7B7D7E808283858788F9
:100540008A8C8E8F91939596989A9C9EA0A2A3A533
:10055000A7A9ABADAFB1B3B5B7BABCBEC0C2C4C634
:10056000C9CBCDCFD1D4D6D8DBDDDFE2E4E7E9EBF0
:10057000EEF0F3F5F8FAFDFF0000000000000000C7
:100580002A2B2800000000000000000000000000EE
:1005900000000029000000002C1E342021222434F9
:1005A0002627252E362D3738271E1F2021222324CB
:1005B00025263333362E37381F0405060708090A67
:1005C0000B0C0D0E0F101112131415161718191A03
:1005D0001B1C1D2F3130232D350405060708090A81
:1005E0000B0C0D0E0F101112131415161718191AE3
:1005F0001B1C1D2F3130354C000000000000000096
:1006000000000000000000000000000000000000EA
:100610000000000000000000000000007E0F00D479
:10062000FFFFFFC7000000781E0353007400650041
:1006300065007A0079003600300020005200650025
:1006400076002000410000000E03340070007000AE
:100650006C006500740000000403090409025B00DB
:10066000030100A0FA0904000001030101000921AF
:10067000110100012244000705810308000109045B
:1006800001000203000000092111010001222200E3
:100690000705820320000107050303200001090468
:1006A00002000103000000092111010001226D0078
:1006B0000705840320000112010002000000084425
:1006C0004402000100010200010660FF0961A1016E
:1006D0000962150026FF009520750881020963153F
:1006E0000026FF00952075089102C005010980A130
:1006F00001850319012AB700150126B70095017578
:10070000108100C0050C0901A101850419012AA06E
:1007100002150126A002950175108100C00501098E
:1007200006A1018506050719E029E71500250195B1
:1007300008750181020507190029EF1500250195AB
:10074000F0750181020508190129059505750191CA
:1007500002950175039101C005010906A101050774
:1007600019E029E715002501950875018102950119
:10077000750881010507190029FF150026FF00955E
:100780000675088100050819012905150025019540
:100790000575019102950175039101C011241FBED9
:1007A000CFEFD4E0DEBFCDBF04B603FE18C080910A
:1007B000950390919603A0919703B0919803873089
:1007C000904BA740B04B59F41092950310929603AA
:1007D0001092970310929803E0E0F8E3099511E076
:1007E000A0E0B1E0EAEBF3E602C005900D92A43F71
:1007F000B107D9F723E0A4EFB1E001C01D92A539FC
:10080000B207E1F70E949A130C94DB310C940000BC
:10081000282F8430E8F46530D8F44E30C8F4862FA1
:1008200090E06EE070E00E94D12FFC01822F90E0FA
:1008300066E470E00E94D12F8E0F9F1FFC01E40F31
:10084000F11DEE0FFF1FE25DFE4F8591949108951B
:1008500081E090E0089581E0089581E008950E948C
:100860002D0408950E942F0408950E942D040895D8
:1008700008950E9438040895A6E0B0E0E2E4F4E0B0
:100880000C947B3049835A839E833091FB0189818C
:100890009A81311115C03E81332359F0222349F04A
:1008A0000E94CD09182F682F89819A810E94A4097E
:1008B00003C00E94B909182F69817A81812F04C071
:1008C0000E94CD0969817A810E943A112696E3E05F
:1008D0000C949730FC01262F4081518162817381F5
:1008E000848195810E943C040895CF93DF93EC01AD
:1008F00061E00E946A04BE010E943204DF91CF9140
:100900000895CF93DF93EC0160E00E946A04BE017A
:100910000E943904DF91CF91089591E001C0990FB1
:100920008A95EAF7892F0E94EE080895CF93C82F81
:1009300081E00C2E01C0880F0A94EAF70E94820E13
:100940008C2F0E948D04CF91089581E008950E941C
:10095000A5040895CF93C82F0E94A0088C2F0E9451
:10096000A7042FEF84E39CE0215080409040E1F702
:1009700000C00000CF91089581E00E94AA040E9467
:10098000D428089580E00E94AA040E94F8280895BF
:10099000A2E0B0E0EEECF4E00C947A308C0161E07F
:1009A0000E946A049A838983F801858181110E94DB
:1009B000911BB801CE0101960E94BE1D882309F447
:1009C00070C0B80189819A810E94AF24882309F4FC
:1009D00068C0B80189819A810E943504882309F48E
:1009E00060C0B80189819A810E94B323882309F4E9
:1009F00058C0B80189819A810E944821882309F44E
:100A000050C0B80189819A810E94941D882309F4FD
:100A100048C0B80189819A810E94B613882309F4DD
:100A200040C0B80189819A810E94F6238823C9F1C8
:100A3000B80189819A810E943812882391F1F801C6
:100A40008581882351F189819A818330FCE79F0752
:100A5000D1F040F48115ECE79E0791F081309C477E
:100A6000A1F01BC08B352CE79207A9F08C35ECE781
:100A70009E0771F08A359C4781F40E945D0E0DC07F
:100A80000E94BC040EC00E94650E0E94C20409C0F0
:100A90000E94530E02C00E94610EC8010E942B04E6
:100AA00001C080E02296E4E00C9496300E94032876
:100AB0000E94760508950E947A050E940C280895E8
:100AC00081E008950895CF93DF93D82F0E946005A9
:100AD000C82F882319F08D2F0E9462058C2FDF917B
:100AE000CF91089508950E946305089580E00E94C3
:100AF000730508950E9428260E9473050895CF93D8
:100B00000E942826C82F8091F601C81779F0C0935B
:100B1000F6010E9493286093F7017093F801809387
:100B2000F9019093FA018C2F0E947305CF910895DB
:100B3000ADE0B0E0EEE9F5E00C947C3048875987F1
:100B40006A877B878C879D8791110E945F0DCE01FC
:100B5000019627E0FC0111922A95E9F726E0FE01B3
:100B60003896DC0101900D922A95E1F72D81211133
:100B70000AC029813A814B815C816D817E818F81A0
:100B80000E94A00C04C00E9475048111F2CF2D9622
:100B9000E2E00C949830FC012481213021F4808122
:100BA00091810E94FA090895CF938823D9F1C82F23
:100BB0008CEF8C0F813A70F48C2F0E94BA26882318
:100BC00029F08C2F0E945F270E94E60D8C2F0E9437
:100BD00045270CC080E28C0F883058F4C77081E044
:100BE00001C0880FCA95EAF70E94420D0E94E60DE7
:100BF00019C0EBE5EC0FE33040F4F0E0EE59FE4FA6
:100C0000808190E00E944E260DC0C85ACB3150F42E
:100C1000EC2FF0E0EE0FFF1FE45DFE4F808191812D
:100C20000E947326CF910895882339F19CEF980F85
:100C3000913A18F40E945F270DC090E2980F983007
:100C400060F4877091E001C0990F8A95EAF7892FC7
:100C50000E94480D0E94E60D08959BE5980F933081
:100C600028F480E090E00E944E260895885A8B3147
:100C700020F480E090E00E94732608951F93CF93A4
:100C8000DF93182FEB010E94D405209741F08FE9E4
:100C90009FE00197F1F700C000002197F6CF812F68
:100CA0000E941406DF91CF911F910895893319F0A6
:100CB00060E070E002C060E570E00E943E060895CA
:100CC000882321F00E94420D0E94E60D089588239A
:100CD00021F00E94480D0E94E60D0895A0E0B0E0CA
:100CE000E4E7F6E00C9476307C01162FC72FFC0168
:100CF000D581068102950F700E94380D8823F9F086
:100D0000DD23E9F08C2F807F803461F080E2810F59
:100D10008830A8F08C2F807E803221F4123078F059
:100D2000002369F08091430382FF09C082E00E94A2
:100D3000270E0E94380D91E0D82ED92601C0D12C63
:100D4000CC2EC2948FE0C8228C2D90E08C3091057F
:100D500008F089C1FC01E65CFF4F0C945F308C2FDA
:100D6000807FCF70882311F0C295C07FDD2399F07A
:100D7000CC2309F464C180E2810F883010F0111196
:100D800004C08C2F0E94420D03C08C2F0E94520D74
:100D90000E94E60D54C1812F0E941406CC2309F451
:100DA00062C180E2810F883038F1112329F18C2F44
:100DB0000E94580D24C08C2F807FCF70803211F09C
:100DC000C295C07F112319F0113099F13CC0809178
:100DD000430382FD17C0DD2349F0CC2329F08C2F7B
:100DE0000E94420D0E94E60D80E02AC180E00E9430
:100DF0001406CC2309F437C18C2F0E94480D0E94A1
:100E0000E60D31C1DD2349F0002309F1013009F07D
:100E10002AC18C2F0E94690D26C1011124C18C2F7B
:100E20000E9467068C2F0E94750D8C2F0E94FA0D70
:100E30001AC1DD2321F0063008F015C108C00530C5
:100E400008F011C115C0DD2331F00111F8C08C2F5D
:100E50000E94600608C1002359F0193309F000C14F
:100E6000FFEF27EE83E0F15020408040E1F7F6C02D
:100E70008C2F0E946706F7C08C2F8695869583700D
:100E800019F0813061F0EFC0DD2321F0812F9C2F1C
:100E9000937002C080E090E00E944E26ECC0DD23FB
:100EA00021F0812F9C2F937002C080E090E00E947F
:100EB0007326E1C08C2F837079F5D111D8C0412FF2
:100EC000429546954770440F440F212F2F70042EF2
:100ED00001C0220F0A94EAF714FF08C08FE090E0E7
:100EE00001C0880F4A95EAF7809501C080E0C69559
:100EF000C695C370822BC23049F058F4C13019F046
:100F00000E94F708B4C00E94F108B1C00E94FD0819
:100F1000AEC00E94EE08ABC0DD2319F08C2F8170AB
:100F200001C08695882309F4A2C0412F42954695B9
:100F30004770440F440F212F2F70042E01C0220F41
:100F40000A94EAF714FF08C08FE090E001C0880F10
:100F50004A95EAF7809501C080E0C695C695C370B2
:100F6000822BC23049F058F4C13019F00E94430975
:100F70007EC00E943D097BC00E94490978C00E9442
:100F8000060975C0CF70DD2339F08C2F0E94180937
:100F9000812F0E9460066BC0812F0E9467068C2FF4
:100FA0000E94240964C0123F21F128F4103F41F04F
:100FB000113FC1F040C0133F19F1143F79F03BC01D
:100FC000DD2341F0053008F04EC08C2F8F710E9458
:100FD000310949C0063008F046C0F7CF809143037D
:100FE00082FD18C0DD2339F08C2F8F710E94180903
:100FF0003AC0DD23C9F38C2F8F710E94240933C0BE
:10100000DD2329F08C2F8F710E940F092CC00E94C4
:101010000B0929C0DD2331F063E08C2F8F710E9412
:10102000090E21C081E00E94270E0230E0F082E02C
:101030000E94270E18C0DD2331F00023A9F2812F72
:101040000E94D40510C00023B1F2193349F49FEF78
:10105000E7EEF3E09150E040F040E1F700C000001F
:10106000812F0E94140688EF8C0D843020F40E949A
:1010700028260E947305DD2089F00E94340D80FD32
:101080000DC0F70115820E942E0D0E941809C7019C
:101090000E946B080E942E0D0E942409CDB7DEB776
:1010A000E8E00C9492300F931F93CF93DF93EC0101
:1010B000688179818D810E94050A8C010E944F0907
:1010C0000E94E108B801CE010E946E06DF91CF9127
:1010D0001F910F910895CF93DF93FC012481222368
:1010E000D1F0EC010E94C80481110FC00E94380D9C
:1010F000882389F08D81882371F08091430382FFDA
:101100000AC082E00E94270E06C0CE010E9453084A
:10111000CE010E948104DF91CF91089580E090E09C
:101120000E944E2680E090E00E9473260E945F0D90
:101130000E94E60D08950E9479270E948E08089566
:101140000E944F0D0E949B08089592959F709630C3
:1011500079F010F4925001C09A50923068F4803FB8
:1011600069F018F4883E40F409C0843F29F406C0B1
:10117000883E20F0813F11F080E0089581E00895DD
:10118000FC012481222339F0808191810E94FA0997
:101190000E94A508089580E00895A6E0B0E0E3ED80
:1011A000F8E00C947C302696E2E00C949830A7E0AE
:1011B000B0E0EDEDF8E00C947C302796E2E00C9482
:1011C0009830089508950E94E20808950E94E30867
:1011D00008950E94E6088093180208950E94E90885
:1011E000089590911802892B0E94E9080895909122
:1011F000180289230E94E90808959091180289270E
:101200000E94E90808950E94E20808950E940309D7
:1012100080931702089580E00E940609089591E0E6
:1012200001C0990F8A95EAF7892F0E94060908954F
:1012300021E030E001C0220F8A95EAF78091170281
:10124000822B0E940609089521E030E001C0220FA0
:101250008A95EAF720958091170282230E94060959
:10126000089521E030E001C0220F8A95EAF78091CD
:10127000170282270E940609089590911702892B70
:101280000E94060908959091170289230E94060979
:1012900008959091170289270E94060908950895DC
:1012A000282FFA01862F8770A1E001C0AA0F8A9526
:1012B000EAF7CB0133E0969587953A95E1F763E03D
:1012C00070E00E94D12FE80FF91F40E050E0622F3C
:1012D00070E090819B01042E02C0369527950A94F8
:1012E000E2F72170219529272A23292721934F5F8F
:1012F0005F4F4330510569F70895FB01A82FA77090
:1013000023E0969587952A95E1F763E070E00E94C7
:10131000D12FE80FF91F40E050E080E0219130E04C
:101320000A2E02C0369527950A94E2F721703327DA
:10133000042E01C0220F0A94EAF7822B4F5F5F4F01
:101340004330510559F70895953090F48E3080F46C
:10135000362F282F892F90E06EE070E00E94D12F69
:10136000BC01620F711D4CEF51E0832F0E945009A8
:101370000895953080F48E3070F4282F892F90E0F6
:101380006EE070E00E94D12F6CEF71E0820F911D32
:101390000E947D09089580E00895CF92DF92FF9228
:1013A0000F931F93CF93DF936C01009117028091ED
:1013B0001802082BC3E0D0E010E0C8010C2E02C0D8
:1013C000959587950A94E2F780FD04C02197A8F7C8
:1013D000F12C07C0FC2EB6018C2F0E9446110197FC
:1013E000A9F38F2DDF91CF911F910F91FF90DF9087
:1013F000CF900895CF93DF93EC010E94CD09BE01F9
:101400000E944611DF91CF9108951F93CF93DF93F0
:10141000EB019091FB01992321F0CB010E94FA0985
:1014200013C0882349F0CB010E94CD09182F682FE3
:10143000CE010E94A40904C0CB010E94B909182F53
:10144000BE01812F0E944611DF91CF911F91089517
:10145000E1E0F0E0DF0102C0AA0FBB1F6A95E2F7EE
:10146000BD01DF0102C0AA0FBB1F4A95E2F7AD0123
:10147000462B01C0EE0F2A95EAF7942F98234913C3
:1014800002C08E2B0895E0958E230895242F462FB9
:10149000682F809117020E94280A0E940609089569
:1014A000CF93DF93C091190280911A02C817A9F057
:1014B000D0E0CE0167E070E00E94D12FFC01E55E34
:1014C000FD4F208131814281538164817581868104
:1014D0000E94D7082196C770E7CFDF91CF9108957A
:1014E000209153023091540240915502509156027E
:1014F0006091570270915802809159020E94D7085A
:101500000895CF93DF938091590282958F7009F0EF
:101510004CC080915802882309F447C020911902D9
:1015200040911A02A0915402B0915302C091550209
:10153000D09156022417C9F130E0C90167E070E08C
:101540000E94D12FFC01E55EFD4F8481882349F183
:1015500081818A1326C080818B1323C085818111EC
:1015600020C0828193818C1B9D0B883C9105C8F41F
:10157000809159028F70806180935902C90167E0A0
:1015800070E00E94D12FFC01EF5DFD4F90819F70B4
:101590009061908383E592E00E946B080E94500A5C
:1015A00004C02F5F3F4F2770C5CFDF91CF910895C3
:1015B000CF93B82FC62F20911902A0911A022A1793
:1015C000B1F030E0C90167E070E00E94D12FFC016A
:1015D000E55EFD4F81818C1306C080818B1303C0B3
:1015E0008581841306C02F5F3F4F2770E8CF80E0CE
:1015F00001C081E0CF910895A4E1B0E0E2E0FBE01A
:101600000C9472308C0186E0F801DE011F96019087
:101610000D928A95E1F7F8018481E58093E5A92E82
:1016200092E0B92E90915702911118C0882309F4C5
:1016300080C1EE20D9F1C8010E94C008F82E88238D
:10164000A9F187E0F801D50101900D928A95E1F7A3
:10165000C5010E94CB050E94810A98C0F801C08094
:10166000D18082809380F090580220915502309171
:101670005602A401421B530BFF2009F406C1483C4B
:10168000510508F0AFC0882309F455C18091590273
:10169000282F207F90915402222361F09D1509F498
:1016A00062C0C8010E94C008811173C0C8010E94B5
:1016B0006B083FC19D1115C0909153029C1111C040
:1016C000E1100FC08F708061809359020E94700AF0
:1016D00083E592E00E946B0880915902F8018683AD
:1016E00026C1E1103AC040E06D2D8C2D0E94D80A31
:1016F00040E06D2D8C2D0E94D80AE82E811117C173
:10170000CF86D88A8F8598890E94FA09292F229539
:101710002F70243020F49F70223028F009C02A5006
:10172000223080F014C0992349F0811107C013C002
:10173000992321F0F8019681907F69F0805E8830CE
:1017400030F409C0803F38F0815F833020F0C80159
:101750000E946B08EF2CFE2CEEC080915902816034
:1017600080935902E4C0909153029C119ACFE110EA
:1017700098CFF8018683C8010E946B0887E0F801C2
:10178000A3E5B2E001900D928A95E1F70E94700AFC
:10179000D2C0EE2009F48ACF20915902822F82957F
:1017A0008F7090E002978CF08091530290915402D8
:1017B000998788879B868A86809157028C871D86A9
:1017C0002E87CE0108960E946B0887E0F801A3E5FA
:1017D000B2E001900D928A95E1F70E94810A0E9481
:1017E000700AA7C090915902292F207FA1F4682D7B
:1017F0009A8A898AA6017A899E2D0E94CD0883E55E
:1018000092E00E946B0887E0F50111928A95E9F752
:101810000E94700A8CC0882309F48DC08091540204
:101820008D1111C0809153028C110DC0E1100BC0BD
:10183000F8019683C8010E946B0887E0F5011192B8
:101840008A95E9F778C0C8010E94C008882309F486
:101850002DCFEE2009F42ACF20915902822F8295B4
:101860008F7090E002970CF4B0CF8091530290916A
:1018700054029A8389839C828B82809157028D8344
:101880001E822F83CE0101969ECF483C510508F061
:1018900040C0882309F44DC0FE2CEE2009F406CF89
:1018A000809154028D1127C0809153028C1123C066
:1018B0009091590290FD16C0892F82958F70282F24
:1018C00030E02115310571F0F80196832F30310594
:1018D00009F451CF8F5F982F9295907F86818F70FA
:1018E000892B48CF87E0F801A3E5B2E001900D9283
:1018F0008A95E1F720C0C8010E94C008811165CF18
:1019000080915902816080935902C8010E946B083E
:1019100012C0682D9A8A898AA6017A899E2D0E9412
:10192000CD0887E0F50111928A95E9F72FCFF12CC8
:1019300002C0FF24F3948F2D6496ECE00C948E305B
:10194000AEE0B0E0E6EAFCE00C947C302887398712
:101950004A875B876C877D878E87CE0108960E94B9
:10196000FC0A882369F06C85662309F45FC028852A
:1019700039854A855B857D858E850E94D70856C04E
:1019800087E0FE013896DE01119601900D928A954E
:10199000E1F76C85662309F449C080911A0290E052
:1019A0009C012F5F3F4F277033274091190250E071
:1019B0002417350709F441C06D8367E070E00E9489
:1019C000D12FDC01A55EBD4F97E0FE01319601905D
:1019D0000D929A95E1F720931A020E94500A26C0B0
:1019E00090E067E070E00E94D12F855E9D4F0E94DD
:1019F000FC0A882379F18091190290E067E070E099
:101A00000E94D12FFC01E55EFD4F20813181428192
:101A100053816481758186810E94D7088091190263
:101A200090E001968770992780931902809119029E
:101A300090911A028913D4CF0DC00E94A008109271
:101A40001A0210921902E3E5F2E087E0DF011D922D
:101A50008A95E9F72E96E2E00C9498308091820204
:101A6000869586958695089580918202877008955F
:101A700090918202977081E009F480E0089580914E
:101A8000AE0208959091AE02892B8093AE02089524
:101A900080959091AE0289238093AE0208951092B2
:101AA000AE0208959091AD02892B8093AD02089506
:101AB00080959091AD0289238093AD020895109294
:101AC000AD02089508950E94620D08950E94630D6D
:101AD000089590918402292F2823821729F0982BAA
:101AE000909384020E94660D089590918402292F9C
:101AF000282331F080958923809384020E94660D0B
:101B0000089580918402882329F01092840280E055
:101B10000E94660D0895CF93C091AE028091AD02F0
:101B2000C82B80918402882331F0C82B0E9498260C
:101B300081110E94810D8C2FCF910895CF93DF9357
:101B4000C0910601D09107010E948B0D8883C0913E
:101B50000601D091070148E050E06AE772E0CE014B
:101B60000E944E31892B59F088E0FE01AAE7B2E0CD
:101B700001900D928A95E1F7CE010E943526DF9102
:101B8000CF910895CF93DF93C0910401D0910501C7
:101B90000E948B0D8983C0910401D091050140E220
:101BA00050E06AE572E0CE010E944E31892B59F077
:101BB00080E2FE01AAE5B2E001900D928A95E1F77C
:101BC000CE010E944026DF91CF9108950E94DC272C
:101BD000813039F48091420387FF03C00E94C20D17
:101BE00008950E949E0D08950E94620D08950E941E
:101BF000F40D089590918302292F282331F08095C8
:101C00008923809383020E94F70D08950E94620D3C
:101C100008959091430392FF11C0982F990F990F47
:101C2000990F692B609382020E94180980918202A9
:101C30008695869586950E94060E08950E9418093D
:101C400008951092820280E00E94060E08959091FD
:101C500082028095892380938202282F277069F45D
:101C6000981759F09091430392FF07C08695869587
:101C700086950E9424090E94210E089590914303A5
:101C800092FB222720F9281769F080FB92F99093A4
:101C9000430380914203909143030E948D0E82E0A2
:101CA0000E94270E08958091430382FB882780F9C4
:101CB00091E089270E943E0E089581E00E943E0E29
:101CC000089580E00E943E0E08956FEF7FEF80E060
:101CD00090E00E94A631089580E090E00E94723169
:101CE000853E9E4F19F40E944124089580E0089596
:101CF00082E090E00E946431089583E090E00E94C9
:101D000064310895682F83E090E00E94883108953F
:101D100084E090E00E9472310895BC0184E090E07C
:101D20000E94A6310895AB01BC018FE090E00E94B3
:101D30009A310895AB01BC0183E190E00E949A3191
:101D4000089560E070E0CB010E949A0E089560E073
:101D500070E0CB010E94930E0E94A10E0895A8E0AE
:101D6000B0E0E5EBFEE00C947C3065EE7EEF80E0C9
:101D700090E00E94A63160E082E090E00E9488310D
:101D800081E0809318020E94820E60E074E184E09A
:101D900090E00E94A63160E086E090E00E948831E9
:101DA00060E087E090E00E94883140E050E0BA01B6
:101DB00088E090E00E949A3160E083E290E00E9427
:101DC000883160E08CE090E00E94883160E08DE036
:101DD00090E00E94883119821A821B821C821D8227
:101DE0001E821F82188648E050E067E170E0CE0155
:101DF00001960E94783140E050E0BA018FE190E016
:101E00000E949A3180E00E945A240E948F240E94EE
:101E1000A70E2896E2E00C9498300E94AF0E089529
:101E2000682F8EE090E00E9488310895A6E0B0E02F
:101E3000ECE1FFE00C947A300E9487288C018091BD
:101E4000AF029091B0020817190781F019821A8227
:101E50000E948728682F49815A81792F80E090E07D
:101E60000E9498051093B0020093AF022696E4E01A
:101E70000C9496300E9493286093BF027093C00226
:101E80008093C1029093C2026093BB027093BC0224
:101E90008093BD029093BE02089581E0089581E091
:101EA00008950E944F0F089508950E94540F0895B9
:101EB0000E94540F08950E94580F08950E94540FD5
:101EC00008950E945E0F08950E94540F089586E3BE
:101ED00092E10E94B1130E94640F0E94610F089565
:101EE0000E94550F0E94540F08950E946C0E81119C
:101EF00002C00E940D0F0E94780E8093C3020E94C0
:101F0000880E90934303809342030E94F41B0E9427
:101F10007D0E0E94EE08809117020E940309089529
:101F20000E947E280E949F240E9409130E94750F20
:101F30000E9472050E949C1A0E945B0F0895A6E001
:101F4000B0E0E5EAFFE00C9470300E944D0F811183
:101F500003C00E94160F62C00E941F1321EBE22EE5
:101F600022E0F22E5701D12CF501019111915F0170
:101F70008D2D0E944B1280279127D394F5E0DF1618
:101F800019F0892B89F302C0892B19F38091C302C0
:101F900081FD0E9454120E94510F782E10E0662499
:101FA0006394812F0E944B124C01F701A080B180F5
:101FB000A826B926A114B10449F100E0CC24C394A9
:101FC000D12CC5018C219D21892BC1F07720B1F046
:101FD00009831A830E9487289C838B836D8221E06A
:101FE000C4018C219D21892B09F420E049815A816B
:101FF0006B817C818D81922F0E9498050F5FCC0CA4
:10200000DD1C0E30F1F6F701918280821F5FF2E055
:10201000EF0EF11C153029F60E943A0F0E94921B18
:102020000E947F052696EEE00C948C301F93CF9390
:10203000DF930E944B11EC01C11580E5D807E8F54C
:10204000C11590E4D90708F0ACC0C03ED10530F509
:10205000CD3CD10508F098C0C83AD10578F4C53A0E
:10206000D10508F087C0C130D10509F480C008F45B
:10207000F9C0C430D10508F0F8C0F4C0C33CD105A4
:1020800008F0F0C0C85AD0E0CC0FDD1FCB59DE4FAE
:102090000990D881C02DCE019464E8C0C11580E2BA
:1020A000D80708F0D2C0C11591E0D90708F06FC079
:1020B000C83ED10508F4D9C0D5C0C03682E5D807DE
:1020C00038F5C03492E5D90708F07DC0C03282E50A
:1020D000D80708F070C0C11592E5D90708F488C088
:1020E0004C2F4695469550E0F5E0440F551FFA9564
:1020F000E1F7C37021E030E0C90102C0880F991FE9
:10210000CA95E2F7EA01C82BD92BCE019D68AEC073
:10211000C03A82E5D807C8F48C2F8F71C03892E599
:10212000D90708F080C08695869590E065E0880F15
:10213000991F6A95E1F7C37021E030E002C0220FD9
:10214000331FCA95E2F73A686BC0C03C82E5D807F6
:1021500008F470C0C03E92E5D90708F083C0CF7183
:10216000DD27DC2FCC27CE01806F906A7FC081E015
:1021700090E07CC0C55AD0E0C556DE4F8881C82F9C
:10218000D0E0CE01906472C0CE0190656FC08D2FFB
:102190000E94E711182FCE0199270E944B111F7141
:1021A0005FC0CE0199270E944B11CC27DF70D06A07
:1021B0008C2B9D2B5BC0CF71D0E0DC2FCC27CE01C8
:1021C000816F906A53C08C2F8F718695869590E0B1
:1021D0009C0175E0220F331F7A95E1F7C37081E00F
:1021E00090E002C0880F991FCA95E2F79C6818C05A
:1021F0008C2F8F710E94E71195E0D695C7959A951F
:10220000E1F7CF70D0E0DC2FCC27282F30E084FF1F
:1022100005C084E0220F331F8A95E1F7D069CE0113
:10222000822B932B23C090E0D82FCC27CE01846F34
:10223000906A1CC08C2F8F710E94E7118F7190E003
:10224000D82FCC27CE01906211C08D2F8F710E94A4
:10225000E711182FCE0199270E944B111F71906230
:10226000912B04C080E090E001C0CE01DF91CF91BE
:102270001F910895753038F46E3028F4462F672F7B
:102280000E94AC1C089580E090E008950E943A11ED
:102290000E94161008958238910569F1B0F48133D7
:1022A000910509F475C048F48932910509F467C0B5
:1022B0008A32910509F471C008958533910509F4B6
:1022C00059C089339105B9F00895833E910589F18C
:1022D00038F4803E9105D1F0823E910529F10895B0
:1022E000863E9105C9F1873E9105D9F1843E91055D
:1022F00009F06CC027C02091420320FD57C021FD8A
:1023000055C02091430323FD5BC008958091420393
:1023100080FD48C08091430380FF48C08091420304
:1023200084FD46C083EE51C08091420382FF3CC0D1
:10233000F5CF8091420382FD37C08091430380FD39
:1023400035C0ECCF8091430381FF36C080914203BA
:1023500084FD2EC087EE39C08091420383FF2AC0DE
:10236000F5CF8091420383FD25C08091430381FD19
:1023700023C0ECCF8091420385FD22C01FC0809115
:10238000420385FD1BC08091430383FF19C00AC02F
:102390008091420386FD16C017C08091420386FDDE
:1023A00013C010C089E311C082EE0FC080EE0DC0D3
:1023B00080E00BC086EE09C084EE07C085E305C04F
:1023C00089E203C08AE201C081E390E00895909120
:1023D000420392FF10C041E0282F2471243009F0FD
:1023E00040E031E0282F2871283009F030E0431711
:1023F00011F02CE0822793FF10C041E0282F2471B8
:10240000243109F040E031E0282F2871283109F00B
:1024100030E0431711F02CE082273091430330FF66
:1024200010C051E0282F2171213009F050E041E027
:10243000282F2871283009F040E0541711F029E0C6
:10244000822731FF10C041E0282F2171213109F08E
:1024500040E031E0282F2871283109F030E043179F
:1024600011F029E0822794FD877E089580E0089589
:10247000CF939C01205E32452032310540F4FB01B0
:10248000C581C11105C08F710E94960401C0C1E0D1
:102490008C2FCF910895E82FF0E0EE0FFF1FE25B45
:1024A000FC4F808191810895089580EA8A95F1F723
:1024B000089500C008950E945512089508950E943D
:1024C0005E1208950E945F1208950E945E120895A0
:1024D0000E9465120895F894E82FE295EF70F0E0FD
:1024E00031A1282F2F7081E090E001C0880F2A953C
:1024F000EAF7982F9095932391A392A1892B82A319
:10250000789408950F931F93CF93DF93CCEAD1E093
:1025100089918F3F11F00E946B1281E0C13BD80777
:10252000B9F7CEE9D1E00CEA11E089918F3F11F0C3
:102530000E946B120C171D07C1F7DF91CF911F91FD
:102540000F910895A0E0B0E0E8EAF2E10C94753054
:102550008C01C62FD0E0CE0184559E4F6C01FC014A
:1025600090819F3F09F450C0B62EF894E92FE29570
:10257000EF70F0E081A19F7021E030E001C0220FF8
:102580009A95EAF7822B81A382A12095282322A382
:1025900078940E945912EEE9F1E04CEA51E021E012
:1025A00030E0E12CF12C61916F3F89F0A62FA295CC
:1025B000AF70B0E090968C9190E06F7002C09595EE
:1025C00087956A95E2F780FD02C0C90102C080E0EC
:1025D00090E0E82AF92A220F331F4E175F0719F7F8
:1025E000F60180818F3F11F00E946B1261E0E114CF
:1025F000F10409F460E08B2D0E945B12CC0FDD1F0B
:10260000C00FD11FF982E882CDB7DEB7E9E00C94A4
:1026100091300E9482128AE0EEE4F3E0DF01982F0D
:102620001D929A95E9F7E4E4F3E0DF011D928A95A3
:10263000E9F785E00E945A130E9468120895AAE003
:10264000B0E0E5E2F3E10C9479308E010F5F1F4FAB
:102650008AE0F80111928A95E9F7F12C6F2DC801F3
:102660000E94A212F394F5E0FF12F8CF4AE050E086
:10267000B80184E493E00E944E3121E0009709F410
:1026800020E0892B41F08AE0F801A4E4B3E0019056
:102690000D928A95E1F745E06EE473E084E493E0FF
:1026A0000E945B13182F0E946212812F2A96E5E088
:1026B0000C9495300895EF92FF920F931F93CF9350
:1026C000DF937C018B01C42F222351F081E08093A2
:1026D000C6020E9487289093C5028093C40204C05A
:1026E0008091C602811102C080E01CC08091C402AA
:1026F0009091C5020E949F280597B0F3D0E0CC0FBF
:10270000DD1FAE01B701C8010E944E31892B39F09F
:10271000AE01B701C8010E945B3181E001C080E0D9
:102720001092C602CDB7DEB7E6E00C9494300E945A
:102730009F0F08950E9424280E947B2A0E94670F01
:102740000E94952A0E94900F0E94A22A0E94A72A06
:102750000E9497130E94C12A0E9455290E94700F5F
:10276000F5CF9093F5018093F40108950F931F9393
:10277000CF93FB01C581CC2309F444C08C010E9496
:102780003F0D8272F801E052F847EB30F105D8F5C1
:10279000EA5BFF4F0C945F300E948E1A27C088239B
:1027A00029F00E947C1A22C08823D9F30E946C1A57
:1027B0001DC0882329F00E94EE1618C08823D9F383
:1027C0000E94DF1613C0882329F00E9410170EC044
:1027D0008823D9F30E94FF1609C0882329F00E949C
:1027E000321704C08823D9F30E942117C0E00BC020
:1027F000882329F00E948A15F9CF8823D9F30E94F3
:102800006A15F4CFC1E08C2FCF911F910F910895DD
:10281000EF92FF920F931F93CF93DF93E82F7111E5
:102820000AC0442321F0F0E0E858FB4FE4916E2FFA
:102830007E2F8E2F6CC0C62FD0E0072F10E0282FE0
:1028400030E0442329F0F901E858FB4F249130E0AF
:10285000CE0166E070E00E94D12FEE24EA94F12CC4
:10286000B7010E941530DB01CC0FDD1FCB016BEAF5
:102870007FEF0E94D12F8C0F9D1FC82FCC0FC80F48
:10288000C701801B910BB9010E94D12FE92F492F5D
:10289000D0E0CE01B8010E94D12F692F70E0C701AE
:1028A000861B970BB9010E94D12FF92FC7018C1BF2
:1028B0009D0BB8010E94D12F692F70E0C701861BC4
:1028C000970BB9010E94D12FA230B10591F040F4CD
:1028D000109761F01197B9F4722F8E2FEF2F16C059
:1028E000A430B10561F040F0169769F4842F792F78
:1028F0000CC0722F892F0AC0822F7F2F07C0822F12
:102900007E2FE92F03C08F2F742FE22F6E2FCDB7AC
:10291000DEB7E6E00C94943041E00E94081408957C
:1029200008950E948C14089590910B01291B922FF9
:10293000E091DE01F091DF01242F462F682F892FCF
:1029400090E009950895CF93DF93762FE901682FE2
:10295000842F0E949114962F672F9E01482F892F54
:102960000E949414DF91CF91089580915803282FED
:102970002695269530E02115310519F48370846081
:1029800005C02B32310524F08370886A8093580388
:102990000895A0E0B0E0EFECF4E10C94763088E02C
:1029A00090E00E946C316B017C0183E290E00E9418
:1029B0006431282F30E040E050E060E070E080E0DB
:1029C00090E000E20E94A330B22FA32FF42FE52F56
:1029D000D62FC72F97018601BC29A12BF22B5E2F82
:1029E000532B2B2F3A2F4F2F6D2F7C2FCDB7DEB7C8
:1029F000E8E00C949230A0E0B0E0E1E0F5E10C9466
:102A0000723049015A016B017C010E94B5148401A6
:102A1000A4016A2D7B2D88E090E00E949A319401F8
:102A20004A2D5B2DB601C70100E20E94BE30622F25
:102A300083E290E00E948831CDB7DEB7ECE00C94E1
:102A40008E30E8E5F3E02081318142815381648159
:102A50007581868197810E94FB140895E8E5F3E073
:102A600025E0208311828FEF828383831482758116
:102A700030E04FEF5FEF60E0868197810E94FB14AA
:102A800008958091580380FF03C086958695089528
:102A900080E00895809158038170089590915C03BF
:102AA000933018F49F5F90935C03882391F02091FA
:102AB00058033091590340915A0350915B03609140
:102AC0005C0370915D0380915E0390915F030E94AF
:102AD000FB14089581E00E944E15089590915C03C7
:102AE000992319F0915090935C03882391F02091E1
:102AF00058033091590340915A0350915B03609100
:102B00005C0370915D0380915E0390915F030E946E
:102B1000FB14089581E00E946E15089580915C0376
:102B2000089580935C03662389F0682F20915803F1
:102B30003091590340915A0350915B0370915D03AA
:102B400080915E0390915F030E94FB14089560E002
:102B50000E949115089580915903089580915A0318
:102B6000089580915B0308950F931F93CF938091F5
:102B7000580380FF09C0E091E201F091E30109955B
:102B8000CF911F910F910895C0910D010091DE0129
:102B90001091DF0180910E01C81768F780910B0139
:102BA0009C2F981B20E040E060E0892F90E0F80126
:102BB0000995CF5FEFCFEF92FF920F931F93CF93C3
:102BC000DF939091580390FF1CC0042F162FD82F2D
:102BD000C0910D01E090DE01F090DF0180910E01C7
:102BE000C81768F480910B019C2F981B202F412F50
:102BF0006D2F892F90E0F7010995CF5FEFCF0E94ED
:102C0000B415CDB7DEB7E6E00C949430909158033C
:102C100090FF0BC0762F682F842F0E948C14962F64
:102C2000672F482F892F0E94DB150895CF93DF93DC
:102C3000EC01EC81F0E0ED58FC4F4491E8E5F3E065
:102C4000628181810E9406168C818F5F8C83DF9167
:102C5000CF910895CF93DF93EC01E8E5F3E0438152
:102C600062818C810E9406168C818F5F8C83DF913C
:102C7000CF910895CF93DF93EC0140915B039C814A
:102C800090FF02C0842F01C080E091FF02C0642F3A
:102C900001C060E092FF40E00E94DB158C8190E073
:102CA0000196877099278C83DF91CF910895A0E0DA
:102CB000B0E0EDE5F6E10C947630182FF62E042FF7
:102CC000E22E9091580390FF6AC0E92FE695E695B1
:102CD000AE2FB0E0AF54BE4F8C9180930C039C7F1D
:102CE000943061F4612F7F2D842F0E948C14962FD5
:102CF000672F482F892F0E94DB153AC0823019F4C4
:102D000000915B0335C0863019F41091590330C02F
:102D10008930D9F3893161F5E9518E2F8170D82E30
:102D2000E695F0E0ED58FB4FE491C12CCE2FD0E0BA
:102D300040910F01C416D0F42C2D30E0C901BE0122
:102D40000E94D12F642F70E00E941530812FD11086
:102D500002C0860F01C0861B90910D01290F311D05
:102D6000402F6F2D0E94A314C394E2CF0E94B4158C
:102D700010935903F0925A0300935B03EE2079F00D
:102D80002091580360915C0370915D03312F4F2DAA
:102D9000502F80915E0390915F030E94FB14CDB78A
:102DA000DEB7E8E00C949230E8E5F3E09181282F5B
:102DB0004381628188E0890F0E945716089581E05F
:102DC0000E94D4160895E8E5F3E09181282F43810D
:102DD000628188EF890F0E945716089581E00E9452
:102DE000E3160895E8E5F3E0628121E1620F08F45B
:102DF0006FEF282F438181810E945716089581E04B
:102E00000E94F2160895E8E5F3E0628121E1621B79
:102E100008F460E0282F438181810E9457160895AD
:102E200081E00E9403170895E8E5F3E0438121E182
:102E3000420F08F44FEF282F628181810E945716BC
:102E4000089581E00E9414170895E8E5F3E04381B6
:102E500021E1421B08F440E0282F628181810E9419
:102E60005716089581E00E942517089520E00E94DA
:102E700057160895EF92FF921F93CF93DF93EC01C3
:102E800010E0EE24EA94F12C60910F011617B8F4CB
:102E900080910D01212F30E0280F311D70E0C70116
:102EA0000E942930812F0E94C82F9C8140915B0392
:102EB00060915A03890F0E94A3141F5FE5CF0E94FF
:102EC000B4159A818C8190FF02C08F5F01C0815040
:102ED0008C83DF91CF911F91FF90EF900895A0E038
:102EE000B0E0E5E7F7E10C947430FC01828180FFEB
:102EF00002C0DFEF01C0D1E0C0E00091DE0110911F
:102F0000DF016CE0A62E80910F01C81708F044C0C5
:102F100080910D0190910B01891B8C0F20E040E006
:102F200060E090E0F801099554E0E52EF12CB12C19
:102F3000CC2ED12C8091C8028B0D8D302CF06A2DB7
:102F40000E940730892F05C087FF03C090910F01B1
:102F5000890F082E000C990BC816D906B1F4809180
:102F60000D019601280F311D80915B0390E0B701A0
:102F70000E94D12F9595879595958795482F6091BB
:102F80005A03809159030E94A314BD0EF1E0EF1A79
:102F9000F10881F6CF5FB7CF0E94B4158091C802C7
:102FA000D13031F4811102C080910F01815007C0EE
:102FB00090E0019660910F0170E00E9429308093AB
:102FC000C802CDB7DEB7EAE00C9490300F931F93A0
:102FD000CF93DF93C0910D010091DE011091DF01CD
:102FE00080910E01C81768F480910B019C2F981BEB
:102FF00020E040E060E0892F90E0F8010995CF5F84
:10300000EFCF10E0C091DE01D091DF0160910F01A0
:10301000161778F5E12FF0E070E0CF010E9429301B
:1030200020910D01820F2091C702022E000C330B5C
:10303000E217F3079CF020910A01022E000C330BDB
:103040002E173F075CF0282F30E040915B03609122
:103050005A03809159030E94A31409C090910B0157
:10306000891B20E040E060E090E0FE0109951F5FD1
:10307000CDCF0E94B415209109018091C702820F23
:103080008093C70290910A01920F90930A0119163A
:103090005CF4082E000C990B40910F0150E0415058
:1030A0005109841795071CF0219520930901DF91A0
:1030B000CF911F910F910895A0E0B0E0E2E6F8E112
:1030C0000C946E308C01FC01C481CC2ED12CE12CEF
:1030D000F12CA7019601C701B6010E94E22FA701BA
:1030E00096010E94E22F4B015C0180E290E06C01AE
:1030F000CC1AD1080D2C000CEE08FF0825E530E0B5
:1031000040E050E0C501B4010E94E22F2B013C01D8
:10311000A7019601C701B6010E94E22FA7019601FF
:103120000E94E22F9B01AC01280D391D4A1D5B1D39
:10313000C301B2010E943D30D22F822F90E02A328B
:1031400030F025E530E0A901481B590BCA0163E0C6
:1031500070E00E94D12F97FD019695958795C82F15
:10316000C095F12C85E5E82EED1A80910F01F81637
:1031700090F4F1FC02C08E2D01C08D2F90910D01B5
:103180002F2D30E0290F311D4C2F60915A030E94E2
:10319000A314F394EACF0E94B415F801848181113D
:1031A00002C091E003C0803219F49FEF90930801B0
:1031B00090910801890FF8018483CDB7DEB7E0E173
:1031C0000C948A300F931F93CF93DF938C01C0E050
:1031D000D0E080910F01282F30E0C217D30734F5DB
:1031E000869590E0F801348120910D01C817D90728
:1031F0003CF4332371F0CE01820F911D9C0106C077
:10320000311107C0FE01E20FF11D9F0140915B03E8
:1032100005C0CE01820F911D9C0140E060915A03D0
:10322000809159030E94A3142196D3CF0E94B41514
:10323000F801848190E00196817099278483DF9161
:10324000CF911F910F910895A0E0B0E0EAE2F9E17B
:103250000C947030FC017280648081E08483E3E729
:10326000F3E08490E2EFF3E0E491C0915B03C69554
:10327000C158D0E0CC0FDD1FCD2EDD24912CAA2427
:10328000AA94B12CE8190E2F10E080910F01981626
:1032900008F096C0E92CF12C82E0871570F0C70188
:1032A00065E070E00E94D12FFC01E753FD4F809153
:1032B0005903808380915A038183C70165E070E0E0
:1032C0000E94D12F611006C0FC01E753FD4F13820D
:1032D000128262C0EC01C753DD4F8B81882321F13C
:1032E00081508B8390E06FEF70E00E94D12F6C8152
:1032F00070E00E941530FB01FF27ED58FC4FE49170
:103300008E2F881990E06FEF70E00E94D12FB801E6
:103310000E94153020915B0330E0862F90E0B901C8
:103320000E94D12F9A8338C00E943131B5010E948A
:1033300029308C159D0584F5E2E0E71588F40E949C
:103340003131B5010E94293088830E9431312091AA
:103350005A032695622F70E00E942930280F298396
:10336000C70165E070E00E94D12F87539D4FFC019B
:10337000128220915B03243120F0293C18F028ECC4
:1033800001C024E1C70165E070E00E94D12FFC017B
:10339000E753FD4F2483238380910D019701280F6C
:1033A000311DC70165E070E00E94D12FFC01E75399
:1033B000FD4F4281618180810E94A314939465CF67
:1033C0000E94B415CDB7DEB7EEE00C948C30E8E582
:1033D000F3E020812E7F20833181428153816481FB
:1033E0007581868197810E94FB1410920D030E94C3
:1033F000B4150895E8E5F3E080818E7F8083109214
:103400000D030E94B4150895609158036695669562
:1034100070E04BE050E080E191E00E944131892B67
:1034200019F481E080930D030E948728909306038E
:103430008093050308959091580390FF3FC09370C7
:10344000811102C0946007C08B3210F0986A03C0EB
:10345000880F880F982B90935803662391F0209142
:1034600058033091590340915A0350915B03609186
:103470005C0370915D0380915E0390915F030E94F5
:10348000FB14609158036695669570E04BE050E040
:1034900080E191E00E944131892B19F010920D03D7
:1034A00002C00E94041A81E08093080340915B03EC
:1034B00060915A03809159030E9436170895682F2E
:1034C000909158039695969581E0890F8B3208F07C
:1034D00081E00E941B1A089581E00E945F1A0895FE
:1034E000682F90915803969596958FEF890F09F460
:1034F0008AE20E941B1A089581E00E94701A0895C2
:1035000061E00E941B1A0895E8E5F3E08081816084
:103510008083869586950E94801A0895809158032D
:1035200080FF03C00E94E71908950E94841A08953D
:1035300060E00E941B1A089580910B0381113CC02A
:103540000E94C914209358033093590340935A039F
:1035500050935B0360935C0370935D0380935E0301
:1035600090935F032C7FA1F40E942E150E94C91432
:10357000209358033093590340935A0350935B03AD
:1035800060935C0370935D0380935E0390935F038D
:103590000E94B51410920D03E091DC01F091DD0161
:1035A00009958091580380FF04C0869586950E94F6
:1035B000981A81E080930B030895E8E5F3E0808199
:1035C00081608083869586950E94981A08958091DF
:1035D000580380FF03C00E94FA1908950E94DD1A63
:1035E00008950F931F93CF93DF9380910D0388234A
:1035F00009F492C080910C03E0915803E695E6959A
:10360000E81BE0930703823049F4F0E0E159FC4FF6
:10361000E491CE2FD0E006E116E159C0863049F49E
:10362000F0E0E459FC4FE491CE2FD0E00AE216E13D
:103630004EC0893051F4E695F0E0E759FC4FE49133
:10364000CE2FD0E00AE317E142C08F3051F4E69567
:10365000F0E0EA59FC4FE491CE2FD0E00FE617E1FD
:1036600036C0853149F4F0E0ED59FC4FE491CE2F9E
:10367000D0E006EE17E12BC08831D9F0833239F45F
:10368000E1E6F3E0C591D4910AE316E120C084326B
:10369000A9F08532C1F48E2F63E00E94FB2FE92F41
:1036A000F0E0E25AFC4FE491CE2FD0E004E219E1C1
:1036B0000EC0C8E2D0E00CE518E109C0C4EFD1E0CB
:1036C00002EE18E104C0C0EDD7E000E914E18091FA
:1036D0000803882361F0109208030E9487289093C2
:1036E00006038093050310920A03109209030E94B7
:1036F0008728E0910503F09106038E1B9F0B8F3FF7
:103700009F4750F4EC0FFD1FF0930603E093050371
:1037100085E093E0F8010995DF91CF911F910F911A
:10372000089508950E94F11A0895539A0895362F26
:1037300063E070E00E94D12FDC01A05ABC4F1196CB
:103740003C9311974C93FD0122830895E0E6F3E04A
:10375000818360834283339693E0E438F907C1F7AD
:1037600008958BB1877F9BB198602FB7F894E0E6FE
:10377000F3E033E0E438F30789F0319148E09BB996
:10378000000000C037FF8BB9330F000000C000C03D
:1037900000C08BB900C04A9591F7EBCF2FBF8FE5E2
:1037A00094E00197F1F700C0000008950E94650EB3
:1037B000089580E00E944B12817008950E941F13AB
:1037C0002FEF86E791E0215080409040E1F700C064
:1037D00000000E941F130E94D91B882321F00E9421
:1037E000D61B0E94D42808950E94DE1B089584E011
:1037F0000895E82F862F90E06CE170E00E94D12FB1
:10380000242F30E0220F331F280F391F8E2F90E016
:103810006CE870E00E94D12F820F931F8896089564
:103820000F931F93CF93DF938430A0F4653090F40F
:103830004E3080F40E94F91B8C010E94643190E0AC
:10384000D82FCC27C80101960E9464319E01282BF5
:10385000C90102C080E090E0DF91CF911F910F91EC
:1038600008950F931F93CF93DF93843080F46530D6
:1038700070F44E3060F4E9010E94F91B8C016D2F49
:103880000E9488316C2FC80101960E948831DF9117
:10389000CF911F910F9108951F93CF93DF93D0E0A5
:1038A000C0E010E0412F6C2F8D2F0E9408049C0176
:1038B000412F6C2F8D2F0E94311C1F5F1E3091F7FE
:1038C000CF5FC53071F7DF5FD43051F7DF91CF9113
:1038D0001F910895EF92FF920F931F93CF93DF9361
:1038E000EA017A01E60EF71E8C01C8018896CE1512
:1038F000DF0569F0003322E0120720F40E946431F2
:10390000888301C0188221960F5F1F4FEECFCDB77D
:10391000DEB7E6E00C949430EF92FF920F931F9382
:10392000CF93DF93EA017A01E60EF71E8C01C801FE
:103930008896CE15DF0559F0003322E0120718F4FF
:1039400068810E94883121960F5F1F4FF0CFCDB75D
:10395000DEB7E6E00C949430843038F4653028F417
:103960004E3018F40E94101C089580E090E00895F5
:1039700080E1089588EA91E00895EF92FF920F9315
:103980001F93CF93DF93EA017A01E60EF71E8C01B5
:10399000C801885A9D4FCE15DF0569F0083A21E02D
:1039A000120720F40E946431888301C01882219696
:1039B0000F5F1F4FEDCFCDB7DEB7E6E00C9494302C
:1039C000EF92FF920F931F93CF93DF93EA017A0157
:1039D000E60EF71E8C01C801885A9D4FCE15DF05F3
:1039E00059F0083A21E0120718F468810E948831E2
:1039F00021960F5F1F4FEFCFCDB7DEB7E6E00C94F7
:103A00009430CF93DF93C8E5D2E060E0CE010E940E
:103A100088312196C11584E0D807B9F7DF91CF919D
:103A20000895A8E0B0E0E7E1FDE10C947230F82ED3
:103A30008FE08F1508F474C08FEF93E00E9464311B
:103A400081116EC008E512E0FF2071F0011594E0CD
:103A5000190709F465C0C8010E946431811101C0D1
:103A6000FA940F5F1F4FF0CFFE0131966F0188E08F
:103A700011928A95E9F77801FFEFEF1AFF0AC80162
:103A80000E94643189831A82882309F449C08130F5
:103A900009F040C0580182E0A80EB11CC7010E9485
:103AA00064318A838823E1F19FEF980F933060F4AB
:103AB000780193E0E90EF11CC5010E9464318B830B
:103AC000882371F11C8226C0843019F54E01E3E091
:103AD0008E0E911C02E010E07501FFEFEF1AFF0A55
:103AE000C5010E946431F40181934F018823C1F024
:103AF0008C3741F4E2E0F0E0EC0FFD1FE00FF11F26
:103B0000108208C00F5F1F4F57010730110521F7C2
:103B100007C0750160E0C6010E94E4228701ABCFB7
:103B20002896ECE00C948E30CF93DF9386319C473F
:103B300009F5EB010E943F0D9D81992371F08A7A6E
:103B400091E009F490E090930E03811102C089E2A4
:103B500001C085E30E94452709C080910E038111B1
:103B600002C089E201C085E30E945F270E94E60D42
:103B700080E001C081E0DF91CF910895A0E0B0E046
:103B8000E4ECFDE10C9472307C01DC01ED91FC91E0
:103B9000CF01815A92454F9720F4B0EAEB27B2E566
:103BA000FB27DB011596CC91CC2309F4B4C2EF3F7F
:103BB000F10579F070F0E935FC4719F010920F0328
:103BC00060C390910F0381E0892780930F03A0E0E9
:103BD00059C3A0910F03AA2309F4EBC010920F035D
:103BE000E03CF10540F4E038F10508F073C0E03442
:103BF000F105D0F505C0EF3FF10509F008F4A0C0CC
:103C000021E030E040E050E060E070E080E090E0F3
:103C10000E2F0E94A330B09110032B2BB0911103F3
:103C20003B2BB09112034B2BB09113035B2BB09144
:103C300014036B2BB09115037B2BB09116038B2BC8
:103C4000B09117039B2B20931003309311034093E3
:103C5000120350931303609314037093150380931E
:103C6000160390931703A1C021E030E040E050E03C
:103C700060E070E080E090E08F01005411090E9444
:103C8000A330B09118032B2BB09119033B2BB091AB
:103C90001A034B2BB0911B035B2BB0911C036B2BB6
:103CA000B0911D037B2BB0911E038B2BB0911F0392
:103CB0009B2B209318033093190340931A035093BE
:103CC0001B0360931C0370931D0380931E0390934A
:103CD0001F036BC021E030E040E050E060E070E0A6
:103CE00080E090E08F01005811090E94A330B0914C
:103CF00020032B2BB09121033B2BB09122034B2BA4
:103D0000B09123035B2BB09124036B2BB09125035F
:103D10007B2BB09126038B2BB09127039B2B2093F9
:103D20002003309321034093220350932303609395
:103D3000240370932503809326039093270335C0B3
:103D400021E030E040E050E060E070E080E090E0B2
:103D50008F01005C11090E94A330B09128032B2B26
:103D6000B09129033B2BB0912A034B2BB0912B032D
:103D70005B2BB0912C036B2BB0912D037B2BB0915F
:103D80002E038B2BB0912F039B2B20932803309372
:103D9000290340932A0350932B0360932C037093C1
:103DA0002D0380932E0390932F03E701F983E8837B
:103DB00069C2E034F105D0F4A0901003B090110373
:103DC000C0901203D0901303E0901403F0901503F9
:103DD000B09116031091170321E030E040E050E06D
:103DE00060E070E080E090E00E2F5DC0E038F1050B
:103DF000E8F4A0901803B0901903C0901A03D09073
:103E00001B03E0901C03F0901D03B0911E03109162
:103E10001F0321E030E040E050E060E070E080E02F
:103E200090E04F01D0E48D1A91083CC0E03CF105D0
:103E3000E8F4A0902003B0902103C0902203D0901A
:103E40002303E0902403F0902503B0912603109102
:103E5000270321E030E040E050E060E070E080E0E7
:103E600090E04F01D0E88D1A91081CC0A090280363
:103E7000B0902903C0902A03D0902B03E0902C032C
